:1000000029C143C142C141C140C13FC13FC13DC1FE
:100010003CC13BC13AC139C138C137C136C135C114
:1000200034C133C132C14368616E6765206C696D4C
:100030006974732E2E2E20202000454550524F4DBE
:10004000204E657720446174612000546F204D611B
:10005000696E20446973706C617920536574204126
:100060006C61726D2054656D7020536574204D6114
:10007000782053575220202053657420506F7765A5
:100080007220416C61726D2046616E204F4E20548B
:10009000656D70202020205265626F6F74202020D3
:1000A0002020202020200053617665203D20202044
:1000B0002B427574746F6E43616E63656C203D20D6
:1000C0002D427574746F6E00535752207761732000
:1000D000746F6F2068696768203D2020004F766547
:1000E000722043757272656E74204661756C74205F
:1000F0002020202000204E6F2053687574646F7795
:100100006E2E202020005365742044656661756C56
:1001100074202020202056616C75657320202020DB
:10012000202020202020005965732F4E6F202B2F78
:100130002D427574746F6E004661696C6564202091
:100140002020202020202020454550524F4D206463
:1001500061746120202020200053797374656D2024
:100160005265626F6F74202020506C65617365204A
:1001700077616974202E2E2E2000507265737320D3
:10018000456E7465722020202020202020005465B8
:100190006D7020697320746F6F206869676800450F
:1001A00072726F7221202020202020202020200029
:1001B00020416D7073202020002046574420524576
:1001C00056205357522043757200574100DF4300B9
:1001D000202020202050412D313030572020202059
:1001E000005265762E322831302E30392E313029AA
:1001F0000054656D702E3A002A0020202020202017
:100200002020202020202020202000436F727265B3
:100210006374696F6E3A004B6F7765727400536157
:1002200076652076616C7565202020202020002DC9
:100230002D2D2D2D2D2D2D2D2D2D2D2D2D2D2D001B
:100240001F171B1D1B171F00303132333435363753
:100250003839300011241FBECFE5D4E0DEBFCDBF5A
:1002600010E0A0E6B0E0ECEAF8E102C005900D92E3
:10027000A636B107D9F710E0A6E6B0E001C01D929E
:10028000AD3BB107E1F71CD90FCBBACE1F920F924D
:100290000FB60F9211248F939F93C098C098C09A65
:1002A000C09AC098C098C09AC09AC09882E08A95B7
:1002B000F1F7C09AC098C09A80916600882329F00F
:1002C000809166008150809366008091670088234A
:1002D00029F08091670081508093670080916800C9
:1002E000882329F080916800815080936800809174
:1002F000B400882329F08091B40081508093B40029
:100300008091B500882329F08091B50081508093B9
:10031000B50080916900882329F08091690081509F
:10032000809369008091B8009091B900C29730F431
:100330008091B8009091B900019602C081E090E0F0
:100340009093B9008093B8008091B8009091B90063
:100350008D9719F481E080936500809184009F91CE
:100360008F910F900FBE0F901F901895E091850010
:1003700080B386958695869521E030E0822781704E
:100380008093A40086B38295869586958370822794
:1003900081708093A50086B31092A60087FD03C0EC
:1003A00081E08093A60080B386958695869580FF30
:1003B00009C086B3829586958695837080FF02C0BA
:1003C000B79950C080B386958695869580FD02C00A
:1003D00091E00AC086B3829586958695837080FFEA
:1003E00002C093E001C092E080917C00882329F450
:1003F00081E080937C009093850080918500E817D0
:1004000049F5F0E0ED55FF4F8081882319F1809187
:100410007D008823F9F480918000882331F480E501
:100420008093B40081E0809380008091B4008823A1
:1004300039F590918000913019F58091B5008823AD
:1004400031F410927F0088E08093B5000895909376
:100450007F00089580918000882391F081E080934F
:100460007D00089510927C0010927D00109285000E
:100470001092800010927E0010927F001092B500C2
:10048000089580936800809168008823E1F70895BB
:100490000895EF920F93982F522F84EA86BF06B6E5
:1004A00007FEFDCF9E7F93B984E886BF06B607FEA0
:1004B000FDCF442379F063B984E886BF06B607FE12
:1004C000FDCF08C0808183B996BF06B607FEFDCF79
:1004D000319605C0852F932F9C01F90194E88E2F4A
:1004E000851B801778F384E986BFEE2039F082E01F
:1004F00080936800809168008823E1F70F91EF9066
:10050000089583B984E886BF06B607FEFDCF089537
:100510000F93982FF901442391F09E7F84EA86BFC0
:1005200006B607FEFDCF93B984E886BF06B607FE80
:10053000FDCF63B984E886BF06B607FEFDCF84EA27
:1005400086BF06B607FEFDCF916093B984E886BFEB
:1005500006B607FEFDCF40E0202F30E021503040AE
:1005600064EC54E812C0842F90E08217930729F4BA
:1005700056BF06B607FEFDCF04C066BF06B607FE2F
:10058000FDCF83B1808331964F5F401760F384E9DC
:1005900086BF0F910895EF92FF920F931F93DF9301
:1005A000CF9300D0CDB7DEB71A82198280E960E020
:1005B00040E09E012F5F3F4F02E0AADF99818A81D0
:1005C000E82EFF24192F00E0E02AF12AFA82E982BE
:1005D000F7FC02C050E007C0882799278E199F09B1
:1005E0009A83898351E029813A81822F8295869569
:1005F0008770843010F440E001C045E0832F9927D4
:1006000087FD9A952AE0829F90011124240F311DC5
:100610003A832983552331F088279927821B930B2E
:100620009A83898389819A818D599F4F24F48DE91A
:100630009FEF9A83898349815A819091A7008AE02C
:10064000989FC0011124481759070CF0C29AC1970E
:10065000481759070CF4C2988091B1002AE0829F94
:10066000C00111244817590724F081E080936F00DE
:1006700002C010926F00CA010F900F90CF91DF91CE
:100680001F910F91FF90EF900895813011F484EC49
:1006900001C084E886BF06B607FEFDCF83B108958A
:1006A000FF920F931F93F0906400F394F092640014
:1006B000EFE8F0E050E087B1807F87B987B1852B04
:1006C00087B940E020E030E0369A3699FECF84B119
:1006D00095B1280F391F4F5F4430B1F736952795F4
:1006E00036952795219331935F5F533021F78091A1
:1006F0009300909194008050924090938B0080934F
:100700008A0097FF04C010928B0010928A002091FB
:100710008A0030918B00C901F3E0880F991FFA9588
:10072000E1F7220F331F820F931F8A599F4F6CEC02
:1007300070E0A7D8FB0170938B0060938A008091D2
:10074000AE0090E0681779071CF081E0809371009B
:1007500080918F00909190009C0173E0220F331FD5
:100760007A95E1F7880F991F280F391F20938F0082
:1007700030939000C90164E470E083D870E0669F14
:10078000C001679F900D769F900D112464E670E084
:1007900064D8062F6093740080919100909192002C
:1007A0009C0153E0220F331F5A95E1F7880F991FE0
:1007B000280F391F2093910030939200C90164E4FF
:1007C00070E05FD870E0669FC001679F900D769FD4
:1007D000900D112464E670E040D8162F60937500E8
:1007E000002309F445C0601758F087EE93E090931A
:1007F0007900809378008091AB008F31A9F53EC0DD
:10080000602F70E0812F90E09C01260F371F681B3E
:10081000790B84E690E0AC01249FC001259F900DE8
:10082000349F900D112419D8CB0105966AE070E031
:1008300014D8709379006093780051E0653F750794
:1008400030F087EE93E090937900809378004091A8
:10085000AB00242F30E080917800909179008217CE
:10086000930760F04F3151F081E08093700006C033
:100870008AE090E0909379008093780085E0F81604
:1008800091F410926400F0938D00E0938C008091BD
:1008900078009091790090937B0080937A00009388
:1008A0007600109377001F910F91FF900895582FB5
:1008B000FB010BC0E199FECF5EBB1FBA81918DBBDE
:1008C000F894E29AE19A78945F5F8E2F861B8417E2
:1008D00088F31EBA1FBA0895582FFB010AC0E19988
:1008E000FECF852F90E09FBB8EBBE09A8DB38193A6
:1008F0005F5F8E2F861B841790F308950F93FC0182
:1009000080917F008823C1F480918500813039F483
:10091000002349F4E617F70764F431960AC08230E1
:1009200059F4002311F0F90104C04E175F070CF4CD
:10093000319781E080937F00CF010F91089510924D
:100940006B0010926C0010926A0081E0809361004D
:10095000089581E0809361000895109261000895E8
:10096000A89589E591E060E840E121E032D789E689
:1009700091E060EC40E121E02CD7FFCF1F9311E024
:100980001093610080916900882389F588E0809345
:10099000690080916A008823A9F48EE192E060E802
:1009A00040E121E016D78AEF91E060EC40E121E0E0
:1009B00010D780916A008F5F80936A008AE08093ED
:1009C000690015C060916A0061548FE292E041E0D5
:1009D00021E0FFD680916A00803130F480916A0076
:1009E0008F5F80936A0003C010936B0002C0109267
:1009F00061001F9108958091B6009091B70060E862
:100A00004FE021E0E6D68AEF91E06FE841E021E097
:100A1000E0D6089587EA90E060E840E121E0D9D689
:100A200087EB90E060EC40E121E0D3D680916E004E
:100A3000882309F044C080917E00882309F088C093
:100A400090918500913081F482E080936D009093C5
:100A50006C001092610090936E0090937F009093D1
:100A60007D0090937E000895923009F071C08091CE
:100A70006300813029F48091B10080939F000DC004
:100A8000823029F48091AB008093A80006C08330A7
:100A900021F48091AE008093AD0081E080937200DC
:100AA00010926B0010926C0010926A0080936100AB
:100AB00080937F0080937D0080937E000895813035
:100AC00009F046C080916B00882309F441C08091F1
:100AD0006300823049F480E468EA70E041E0E7DED8
:100AE0008091A8008093AB0080916300813049F42D
:100AF00088E06FE970E041E0DADE80919F0080934A
:100B0000B10080916300833049F487E06DEA70E0C2
:100B100041E0CDDE8091AD008093AE008091630016
:100B2000843049F483E063EB70E041E0C0DE809103
:100B3000B3008093A70081E08093720010926B0055
:100B400010926C0010926A008093610010926E0007
:100B5000089551DF87E291E060EC40E121E039D671
:100B600080917E008823A1F480918500813019F462
:100B700080937E00F5DE80918500823049F481E02B
:100B800080937E008093720080937F0080937D002D
:100B900008950F931F9389EB91E060E840E121E015
:100BA00018D60AEC11E0C80163EC41E021E011D64F
:100BB000C80167EC41E021E00CD6C80101966FEC5A
:100BC00041E021E006D61F910F91089580918400A5
:100BD000882319F010928400DCDF0895809184004E
:100BE000882319F08AE390E002C086E290E060E892
:100BF00040E121E0EED58EE890E060EC41E020E0BD
:100C0000E8D58091B6009091B70061EC4FE021E00B
:100C1000E0D580917F00882391F580918500813017
:100C200091F480916300853048F48F5F8093630076
:100C30008091B6009091B7000F9619C01092630092
:100C40008BE490E014C08230D1F48091630088235B
:100C500049F08150809363008091B6009091B70075
:100C60000F9705C085E08093630086E990E090933C
:100C7000B7008093B60081E080937F000895809153
:100C80007E00882351F580918500833031F5809175
:100C900063008230B1F0833028F4882351F0813032
:100CA000C9F40DC0843089F0843068F0853091F447
:100CB0000EC01092720081E033D56BDF0BC08BE069
:100CC00007C08CE005C08DE003C08EE001C08FE05E
:100CD0008093720081E080937E00089581E020D5AA
:100CE00080ED91E060E840E121E073D581EE91E094
:100CF00060EC40E121E06DD5A8958DE78093680018
:100D0000809168008823E1F7A8958DE780936800BB
:100D1000809168008823E1F7A89581E001D50895C6
:100D2000DF92EF92FF920F931F93DF93CF9300D048
:100D300000D000D0CDB7DEB7FC01162FD22E8091A7
:100D40006C00882329F080916100882309F49AC0FF
:100D5000F7FF07C081E080938300F095E195FF4F96
:100D600002C010928300CF0160E177E28AD5062F9E
:100D7000CF0160E177E285D59C0168EE73E081D513
:100D8000F62EC90168EE73E07CD59C0164E670E044
:100D900078D5E62EC90164E670E073D59C016AE05F
:100DA00070E06FD5E82FF0E0E85BFD4FE491EE8353
:100DB000C9016AE070E065D5E62FF0E0E85BFD4F21
:100DC000E491ED83EE2DF0E0E85BFD4FE491EC83E0
:100DD000EF2DF0E0E85BFD4FE491EB83E02FF0E0D6
:100DE000E85BFD4FE491EA83002311F090E003C03B
:100DF00080E28A8391E0FF2029F4002319F480E245
:100E00008B839F5FEE2039F4FF2029F4002319F42F
:100E100080E28C839F5F809183008130A1F49130C8
:100E200049F0913028F0923041F0933081F408C0BD
:100E30008DE20CC08DE28A830AC08DE28B8307C0ED
:100E40008DE28C8304C0992311F480E28983242FDE
:100E500030E0CE010196DD2069F0821B930B141B5C
:100E600041500696612F20E0B4D48EE29AD48E8150
:100E700098D408C01F5F821B930B141B0696612F2A
:100E800020E0A7D426960FB6F894DEBF0FBECDBFE4
:100E9000CF91DF911F910F91FF90EF90DF90089518
:100EA00081E08093610080918A0090918B0065ECD5
:100EB00042E020E035DF80916900882389F58FE9E1
:100EC00091E060E847E021E084D48DED90E067E8B0
:100ED00049E021E07ED486EE90E060EC44E021E041
:100EE00078D48AEE90E066EC4AE021E072D48091FA
:100EF0006A00813049F48AEF91E060E847E021E040
:100F000068D410926A0009C080916A00882341F475
:100F100080916A008F5F80936A0082E3809369000A
:100F200010926100089581E08093610080917800C3
:100F3000909179006FEC43E021E0F2DE809169004E
:100F4000882359F58FE991E060E848E021E041D439
:100F500088EC90E068E848E021E03BD480ED90E048
:100F600060EC4CE021E035D480916A00813049F496
:100F70008AEF91E060E848E021E02BD410926A000B
:100F800009C080916A00882341F480916A008F5FD4
:100F900080936A0082E38093690010926100089553
:100FA00081E080936100F7DA6DE844E021E0B8DE8B
:100FB0008DEC91E06EE842E021E00BD48091690075
:100FC000882329F58FE991E060E849E021E001D428
:100FD0008EE891E060EC40E121E0FBD380916A0073
:100FE000813049F48AEF91E060E849E021E0F1D3F3
:100FF00010926A0009C080916A00882341F48091B0
:101000006A008F5F80936A0082E380936900109288
:10101000610008950F931F93182FC19A81E0809368
:101020006C0002E0163631F0173631F0153629F42F
:10103000B7DF03C078DF01C033DF98D9A8950093EC
:101040006800809168008823E1F780917E00882302
:1010500049F780918500833029F781E080937E00F5
:101060001092720010926B0010926C0010926A0045
:1010700080936100C19854D38CDD1F910F91089526
:101080000F93B9DC8AEF91E060EC45E021E0A1D359
:101090008DEC91E068EC42E021E09BD38AEF91E097
:1010A0006AEC46E021E095D38091B300873C89F457
:1010B0008FE292E065EC43E021E08BD38091B300B6
:1010C00090E064E670E049E150E028E230E001E0C1
:1010D0000FC090E067EC43E020E022DE8091B30097
:1010E00090E064E670E049E150E020E030E000E0AC
:1010F00005DC8093B30080917E00882351F48091B9
:101100008500833031F481E080937E0084E1809318
:1011100072000F9108950F936EDC8AEF91E060ECFE
:1011200045E021E056D380EB91E068EC48E021E017
:1011300050D38091AD00813B89F48FE292E065EC61
:1011400043E021E046D38091AD0090E064E170E09F
:1011500042E050E02FE030E001E00FC090E067ECAB
:1011600043E020E0DDDD8091AD0090E064E170E0DF
:1011700042E050E020E030E000E0C0DB8093AD00D2
:1011800080917E00882351F480918500833031F472
:1011900081E080937E0084E1809372000F91089536
:1011A0000F9329DC8091A8008C3BE9F48FE292E058
:1011B00065EC43E021E00DD38AEF91E060EC45E07F
:1011C00021E007D38AEF91E068EC48E021E001D309
:1011D0008091A80090E06FE170E04CE050E02FE0DB
:1011E00030E001E026C08F3139F485EF90E060EC0B
:1011F00040E121E0EED213C08AEF91E060EC45E0DF
:1012000021E0E7D28AEF91E068EC48E021E0E1D20A
:101210008091A80090E067EC43E021E081DD8091BF
:10122000A80090E06FE170E04CE050E020E030E09A
:1012300000E064DB8093A80080917E00882351F455
:1012400080918500833031F481E080937E0084E1D9
:10125000809372000F9108950F93CDDB8AEF91E098
:1012600060EC45E021E0B5D28DEC91E068EC42E025
:1012700021E0AFD28AEF91E06AEC46E021E0A9D20A
:1012800080919F00873C89F48FE292E065EC43E017
:1012900021E09FD280919F0090E064E670E049E1F8
:1012A00050E02BE430E001E00FC090E067EC43E059
:1012B00020E036DD80919F0090E064E670E049E137
:1012C00050E020E030E000E019DB80939F00809147
:1012D0007E00882351F480918500833031F481E0D1
:1012E00080937E0084E1809372000F91089588E0DE
:1012F00082BB97E091BB8AEF88BB97BB15BA14BA43
:1013000081E180B91EBC87E28BBD80E18ABD8EB5CC
:1013100081608EBD8EB588608EBD89B7806189BFC2
:1013200081B5886181BD81B5876081BD81B58860E7
:1013300081BD789412D280E492E060E072D23E9A4D
:1013400083E886B9369A3699FECF84B195B188E0A4
:1013500061EB70E041E0C0DA9091B100892F8951D2
:101360008C3458F081E08093AF008093840087EC48
:1013700080939F008093B10004C090939F001092CF
:10138000AF0083E067EA70E041E0A6DA9091A70041
:10139000892F89518C3458F081E08093BA00809372
:1013A000840087EC8093B3008093A70004C09093DF
:1013B000B3001092BA0080E46BEA70E041E08CDA8E
:1013C0009091AB00892F8C50843158F081E080934C
:1013D000B000809384008CEB8093A8008093AB00D6
:1013E00004C09093A8001092B00087E06EEA70E00D
:1013F00041E072DA8091AE00853158F081E080934F
:10140000A9008093840081EB8093AD008093AE00AF
:1014100004C08093AD001092A90080B38695869594
:10142000869580FD0DC086B38295869586958370DE
:1014300080FD06C0B79904C081E0809373001CC092
:1014400080918400882369F088E391E060E840E1BE
:1014500021E0BFD188E491E060EC40E121E0B9D126
:10146000FFCF109272003ADC94DB95D89093A100E4
:101470008093A000C198089579D786E091E060E854
:1014800040E121E0A6D186E191E060EC40E121E07D
:10149000A0D180918500882379F720DC7ADB7BD886
:1014A0009093A1008093A00021E0209372008AE530
:1014B00090E09093B7008093B60020936300089566
:1014C000EF92FF920F931F93CF93DF9310DF16E0FD
:1014D000E12ECAE5D0E009E1B8E7FB2EA89580919E
:1014E0006C00882329F080916D00823009F446DA7F
:1014F000809173008823B1F480916F00882311F0EC
:1015000085E688DD80917000882321F086E682DD03
:101510001092700080917100882321F087E67ADDB7
:101520001092710080916600882309F0B6C0E092A5
:101530006600B6D81BD7809172008D30B1F08E3026
:1015400038F48B3071F08C3070F48130A9F407C01E
:101550008F3079F08F3058F0843171F40CC03EDB5D
:101560000BC07ADE09C01CDE07C0D5DD05C088DDF2
:1015700003C0EFDA01C04EDA80917200882309F0CF
:101580008CC0109162001130E9F58091760090E0F6
:1015900062EC43E020E0C4DB8091770090E066ECF1
:1015A00043E020E0BDDB80918C0090918D006EECDB
:1015B00042E020E0B5DB80917A0090917B006BECFB
:1015C00043E021E0ADDB80917E008823D9F4909147
:1015D0008500913031F482E08093620090937E0028
:1015E00011C0923019F4909362000AC0933051F404
:1015F00010937200D093B700C093B60010936300AD
:1016000010937E0080916200823009F046C081EF25
:1016100091E060E846E021E0DCD08091A00090916C
:10162000A1006AE844E021E07BDB8DEC91E06BE80F
:1016300042E021E0CED08AEF91E06DE843E021E086
:10164000C8D08AEF91E060EC40E121E0C2D0809107
:101650007E00882311F510918500113029F4109334
:10166000620097DA10937E0080918500823031F419
:1016700011E0109362008DDA10937E008091850056
:10168000833059F481E080937200D093B700C09307
:10169000B6008093630080937E008091670088236A
:1016A00009F01CCF0093670076D79093A100809338
:1016B000A00080917200882309F010CF8091600013
:1016C000882321F081508093600008CFF092600061
:1016D00044D080E492E060E0A4D05BDAFFCE81B336
:1016E0008F7081BB82B3806F82BB9098919A20E00B
:1016F00030E02F5F3F4F83E0283E380769F0929A31
:10170000929A929A929A80B392989298929892987A
:10171000929A929887FDEDCF81B3806F81BB089537
:10172000282F9098919882B38F7082BB92B3822FAA
:10173000807F892B82BB929A9298283369F02F324E
:1017400051F082B38F7082BB82B32295207F822BAF
:1017500082BB929A9298C3DF08950F931F9381B32F
:10176000806F81BB929888E3DBDF04EC19E0C8014D
:101770000197F1F788E3D4DFC8010197F1F788E317
:10178000CFDFC8010197F1F78FE2CADF88E2C8DF37
:101790008CE0C6DF81E0C4DF86E0C2DF1F910F91DD
:1017A0000895909A919892B39F7092BB22B3982F0C
:1017B000907F922B92BB929A929892B39F7092BB19
:1017C00092B38295807F982B92BB929A929887DFF2
:1017D0000895EF92FF920F931F93CF93DF938C01A5
:1017E000E42EF22E80916C00882321F0809161001C
:1017F000882381F0862F94DFE80108C0FF2019F0CC
:10180000FE01849101C08881CCDF21969E01201BBE
:101810002E15A0F3DF91CF911F910F91FF90EF90C4
:1018200008950F931F93CF93DF938C01862F880F1A
:10183000880F880F806474DFC0E0D0E0F801EC0FFF
:10184000FD1FE4918E2FADDF2196C830D105B1F791
:10185000DF91CF911F910F910895AA1BBB1B51E1FE
:1018600007C0AA1FBB1FA617B70710F0A61BB70B10
:10187000881F991F5A95A9F780959095BC01CD01B5
:10188000089597FB092E07260AD077FD04D0E5DFDF
:1018900006D000201AF4709561957F4F0895F6F7F1
:0C18A000909581959F4F0895F894FFCF1C
:0618AC003B0101010301F4
:00000001FF
